:10000000B601E329B616B61EB612B6190B28B615F8
:100010004620031832280830A3005B20A20DA30B52
:100020000D28B61E3D2065206120B61A32203720EB
:1000300022080310DE29B616B61EB6123619252878
:10004000FE39B70036150310DE29361A2D28A60012
:10005000361646200318322826084E200318322868
:10006000B61EDE293D20652036113612B6113A083B
:10007000840038088417800443283A08840038092B
:1000800080058417800544284528DE29372065200F
:10009000E2213D2061203708B6190138A20008305E
:1000A000A300A20D03183720031C3D20652061200A
:1000B000A30B5128372065203A0884003808000532
:1000C000FF3E3B088400390940283B08840039087A
:1000D0003A28A400B7172730A30010307B20033044
:1000E000A300E8307B20A30164307B20A3010A3009
:1000F0007B2024088628A2002508A1002408A0004F
:10010000AC212008031DB713B71B0800303EA70021
:100110000711871087108316071187108710F0309A
:10012000860583122708B618B3283A30A100983004
:1001300087213330A600C8201330A10088308721E2
:10014000C82064308621C820643086212230A60071
:10015000C8202830B2200C30B2200630B220B614AD
:100160002708B3283614A600361CC1288710033C84
:10017000031CC628C6200730A100D03087210314F5
:1001800008003614FE3C0319DE298714A60E361C1F
:1001900036100715F030860526080F39860407113A
:1001A000A60E3618C8283230862103140800B8007D
:1001B000841780048413A201201CA200E5200319E7
:1001C000DE29E5200319DE29E5283808A2060130DA
:1001D000A000A101000838052206031D0800A00A9E
:1001E0000319A10FEA280800A501A400B7172730BA
:1001F000A300103007210330A300E8300721A3013A
:1002000064300721A3010A30072124081229A20023
:100210002508A1002408A000AC212008031DB71365
:10022000B71B0800303EA6003A0884000930A7003A
:1002300003101F21A60CA70B192903141F298413CF
:10024000B71D2E2900083804371D38068000841792
:1002500000083804031C38068000392900083804D7
:10026000031C3806371938068000841738098005C2
:100270003929370D0639A0004221A100A00A4221E8
:100280000000872901308A00200882070134993450
:1002900003343934003460340C34FD34A000A00D34
:1002A000A00DA00D3830A005813020049F00003043
:1002B000A100323087211F151F195C291E08A100DB
:1002C00083161E08DE2903178D0083168C130C1469
:1002D00083120C08DE2903178C0083168C130C156F
:1002E00055308D00AA308D008C148C1875290C1196
:1002F000DE29A301A200FF30A207031CA307031CF1
:10030000DE290330A100E73087217B29A101FC3ED3
:10031000A000A109031C9229FF300000A0070318C8
:100320008D29A0076400A10F8C290800A2000130CC
:100330009C29A20006309C29A80023082102031D45
:10034000A3292208200204300318013003190230C7
:100350002805031DFF30DE291030A600A501A401E9
:10036000210DA40DA50D2208A4022308031C230FB0
:10037000A5020318C2292208A40723080318230F83
:10038000A5070310A00DA10DA60BB0292008DE299A
:100390001030A800A101A001A70CA60C031CD629AF
:1003A0002208A00723080318230FA107A10CA00C03
:1003B000A50CA40CA80BCC292408DE298313031355
:1003C0008312640008008316DF30850085309F00AB
:1003D00070308600811387018312850186018701B1
:1003E0000710831607106430831279218A11AB2A13
:1003F000861783168613FE308312872001308720EC
:1004000048308720653087206C3087206C3087200B
:100410006F30872020308720213087200330A300D1
:10042000E8307A21FE30872001308720563087203F
:100430003130872043308720323087204930872071
:100440005230872020308720763087206530872003
:10045000723087202E308720373087202F3087203A
:1004600032308720303087200130A300F4307A21E9
:10047000FE308720C0308720B1308720B5308720FC
:10048000203087206B3087206530872079308720A7
:1004900020308720743087206F30872020308720DD
:1004A0005330872074308720613087207230872056
:1004B000743087206400061B5A2A08000130A0000F
:1004C000053084000430D7202008C8002108C90066
:1004D000080000304E21BC002108BD000A307921FF
:1004E000080001304E21BE002108BF000A307921EA
:1004F00008000730BA001030B8000730BB000830E1
:10050000B900A0301D2041081D2040081D203F08D3
:100510001D203E081D2043081D2042081B200A30D4
:10052000792108000730BA001030B8000730BB004E
:100530000830B900A0301D2041081D2040081D20B2
:100540000420BF000420BE000420C3000220C2001B
:100550000A30792108008613831686138312F82146
:100560000330A300E8307A21FE3087200130872055
:10057000B1308720B53087203A3087204C30872033
:100580006F3087206730872020308720B730872062
:10059000203087203A308720503087206C308720E9
:1005A0006130872079308720FE308720C030872057
:1005B000B1308720B63087203A3087204C308720F2
:1005C0006F30872067308720203087205330872086
:1005D000743087206F308720703087200130A3006F
:1005E000F4307A2164008A11061F092B8A118617BC
:1005F0008316861332308312792164008A11861E95
:10060000122C8A11861383168613323083127921B5
:10061000F22ACC0164000A304C028A110318242B00
:100620008A1186138316861383120130A300F430D7
:100630007A2186178316861383120130A300F430C3
:100640007A21CC0A031D0A2BC001C1014008A00079
:100650004108A1001F30A3003F3096218A11031DDD
:10066000B92B8A114008A0004108A1000430A20063
:10067000A301AC21B2002108B30001303207C4004D
:1006800033080318013EC50071225E220310480D95
:10069000C200490DC30064008A11051A562B8A1145
:1006A0003030C20775300318013EC307FE30872083
:1006B0000130872044308720233087203D30872039
:1006C0004508A50044086920FE30872002308720B5
:1006D000FE30872014308720FE308720143087209A
:1006E000FE30872014308720FE308720143087208A
:1006F000FE30872014308720FE308720143087207A
:10070000FE30872014308720FE3087201430872069
:10071000FE308720143087203F08A5003E0869205E
:10072000303087206D30872056308720FE3087207C
:10073000C0308720433087204830872032308720E0
:100740003D3087204308A500420869207530872086
:100750005330872079224630792164008A11061EA1
:10076000BA2B8A110430C007031C262BC10A031DB3
:10077000262BB42A86138316861383120130A30016
:10078000F4307A214008CB004008A0004108A100C5
:10079000A2010130A300AC21CA00031705308D006F
:1007A00003134B086B21031706308D0003134A080F
:1007B0006B21FE3087200130872053308720743032
:1007C00087206F308720703087204C3087206F3033
:1007D00087206730872067308720693087206E3018
:1007E000872067308720FE308720C0308720453043
:1007F00087204E3087204430872020308720543097
:100800008720493087204D308720453087203D3074
:1008100087204508A500440869201330A3008830CC
:100820007A21B42A861783168613FE308312872016
:1008300001308720B1308720B53087203A308720BB
:10084000503087206C3087206130872079308720B6
:1008500020308720B7308720203087203A3087200B
:100860005330872074308720653087207030872090
:10087000FE308720C0308720B1308720B6308720F7
:100880003A308720453087204E30872044308720FB
:100890000330A300E8307A2164008A11061F572C28
:1008A0008A1164008A11861E792D8A114C2C8613B8
:1008B00083168613053083126321CB000630632133
:1008C000CA004A08A600A701A2010130A300C8215E
:1008D000B2002508B3004B083207C60033080318DE
:1008E000013EC700C001C1014008A0004108A100AD
:1008F0004708A300460896218A11031D352D8A1149
:100900004008A0004108A1000430A200A301AC21CE
:10091000B2002108B30001303207C40033080318C5
:10092000013EC5009222FE308720013087204430EE
:100930008720233087203D3087204508A5004408C4
:100940006920FE30872002308720FE308720143057
:100950008720FE30872014308720FE308720143017
:100960008720FE30872014308720FE308720143007
:100970008720FE30872014308720FE3087201430F7
:100980008720FE30872014308720FE3087201430E7
:1009900087203F08A5003E086920303087206D3051
:1009A000872056308720FE308720C0308720433094
:1009B000872048308720323087203D308720430809
:1009C000A500420869207530872053308720073002
:1009D000BA004030B8000230B70044301321613013
:1009E00013217430132161301321233013213D3042
:1009F00013212C3013214508A5004408F5202C3084
:100A0000132141301321303013213D3013212C307C
:100A100013213F08A5003E08F520303013212C306B
:100A200013216D301321563013213A3013214330F6
:100A3000132148301321323013213D3013212C3043
:100A400013214308A5004208F5200D3013210A3078
:100A5000132164008A11061E3A2D8A110430C00742
:100A6000031C742CC10A031D742C0730A300D03062
:100A70007A21B42AFE308720013087205330872026
:100A8000743087206F308720703087202030872097
:100A9000503087206C308720613087207930872064
:100AA0006230872061308720633087206B30872059
:100AB000FE308720C0308720453087204E30872089
:100AC00044308720203087204430872061308720C1
:100AD0007430872061308720233087203D30872085
:100AE0004508A500440869200B30A300B8307A21DE
:100AF000B42A861383168613053083126321CB0034
:100B000006306321CA004A08A600A701A2010130ED
:100B1000A300C821B2002508B3004B083207C60065
:100B200033080318013EC700C001C1016400861EDE
:100B3000962D4008A0004108A1004708A3004608E0
:100B400099218A11031DA72D8A11C001C1014008F6
:100B5000A0004108A1000430A200A301AC21B20012
:100B60002108B30001303207C40033080318013EE6
:100B7000C5009222FE308720013087204430872034
:100B8000233087203D3087204508A5004408692090
:100B9000FE30872002308720FE30872014308720E7
:100BA000FE30872014308720FE30872014308720C5
:100BB000FE30872014308720FE30872014308720B5
:100BC000FE30872014308720FE30872014308720A5
:100BD000FE30872014308720FE3087201430872095
:100BE0003F08A5003E086920303087206D308720FF
:100BF00056308720FE308720C03087204330872042
:100C000048308720323087203D3087204308A500B8
:100C10004208692075308720533087200730BA009A
:100C20004030B8000230B700443013216130132146
:100C30007430132161301321233013213D301321EF
:100C40002C3013214508A5004408F5202C30132131
:100C500041301321303013213D3013212C3013212A
:100C60003F08A5003E08F520303013212C30132119
:100C70006D301321563013213A30132143301321A4
:100C800048301321323013213D3013212C301321F1
:100C90004308A5004208F5200D3013210A30132126
:100CA00064008A11861A5E2E8A110430C002003058
:100CB000031C013EC102C8307921992D64008A11BC
:100CC000061E702E8A1164008A11061B6F2E8A116F
:100CD0000430C0070318C10AC8307921992D502E5D
:100CE000FE308720013087205330872074308720E2
:100CF0006F30872070308720203087205030872049
:100D00006C308720613087207930872062308720DF
:100D100061308720633087206B3087200730A30045
:0A0D2000D0307A21B42A6300932E2C
:02400E00763DFD
:00000001FF
